:03000000022B9C34
:0C2B9C0078FFE4F6D8FD75816C022BE395
:100E29000A53746172743A20004950436F6E6E65BB
:100E390063745245510A004950436F6E6E6563747D
:100E4900003E432C562C52432CC0E4E0EFF2E5F06F
:100E590020D1E8EDEAEEEC49500A003E432C4D4121
:100E6900432C25303262583A25303262583A2530BF
:100E79003262583A25303262583A25303262583A4D
:100E890025303262582C4D414320E0E4F0E5F10A67
:100E9900003E432C5645522C20332E3120EEF220B1
:100EA90025732025732CC2E5F0F1E8FF2049502075
:100EB900ECEEE4F3EBFF0A004A616E203330203296
:100EC9003030380031313A31383A3332003E432C30
:100ED9004C442C50524F473A2020202020202020DB
:100EE90020202020202020202020202020202020F9
:100EF90020202020202020202020202020202020E9
:100F090020202020202020202020202020202020D8
:100F1900202020202020202020202020202CC4E058
:100F2900F2E020EFF0EEF8E8E2EAE828F4E0E9EB95
:100F3900290A003E2A2C312CCEF1EDEEE2EDFBE53B
:100F490020EFE0F0E0ECE5F2F0FB20F1E5F2E5E27C
:100F5900EEE3EE20E8EDF2E5F0F4E5E9F1E00A0070
:100F69003E412C4130312C2562752E2562752E2586
:100F790062752E2562752C495020E0E4F0E5F120D8
:100F8900E0E4E0EFF2E5F0E00A003E412C413032C6
:100F99002C2562752E2562752E2562752E256275A2
:100FA9002C495020E0E4F0E5F120EEF1ED2E20F19E
:100FB900E5F0E2E5F0E00A003E412C4130332C2512
:100FC90062752E2562752E2562752E2562752C494E
:100FD9005020E0E4F0E5F120F0E5E72E20F1E5F01E
:100FE900E2E5F0E00A003E412C4130342C256275DF
:100FF9002E2562752E2562752E2562752CCCE0F1A1
:10100900EAE020F1E5F2E80A003E412C4130352CB6
:101019002562752E2562752E2562752E2562752C21
:10102900D8EBFEE70A003E532C4130362C25627579
:101039002CC2F0E5ECFF20EEE6E8E42E20EAE2E837
:10104900F2E0EDF6E8E820282A3130ECF1290A002F
:101059003E2A2C312CC4EEEF2E20EFE0F0E0ECE537
:10106900F2F0FB20F1E5F2E5E2EEE3EE20E8EDF245
:10107900E5F0F4E5E9F1E00A003E422C5330312C69
:101089002562752CC6E4E0F2FC20E7E0EFF0EEF112
:10109900E020F1EEE5E4E8EDE5EDE8FF20EEF220F1
:1010A900F1E5F0E2E5F0E00A003E422C5330322C43
:1010B9002562752CCEE1ECE5ED20F120F1E5F0E2B9
:1010C900E5F0EEEC20E1E5E720EAE2E8F2E0EDF612
:1010D900E8E90A003E422C5330332C2562752CCFA7
:1010E900E5F0E5E7E0EFF3F1EA20EFF0E820EFEED5
:1010F900F2E5F0E520F1E2FFE7E820F120F1E5F083
:10110900E2E5F0EEEC0A003E422C5330342C256225
:10111900752CCDE5F220EFE5F0E5E4E0F7E820E411
:10112900E8E0E3EDEEF1F2E8EAE820E220F1E5F0AB
:10113900E2E5F00A003E422C5330352C2562752C2D
:10114900CAE0EDE0EB20F8E8F0EEEAEEE2E5F8E0DF
:10115900F2E5EBFCEDEEE3EE20EEE1ECE5EDE00A85
:10116900003E532C5330362C25303262582530320C
:101179006258253032625825303262582530326241
:101189005825303262582C4D414320E0E4F0E5F116
:1011990020F8E8F0EEEAEEE2E5F8E0F2E5EBFCED46
:1011A900EEE3EE20EEE1ECE5EDE00A003E454E44CB
:1011B9000A0044756D7058202020202030302030DE
:1011C9003120303220303320303420303520303651
:1011D900203037203038203039203041203042202B
:1011E90030432030442030452030460A003A003A46
:1011F90020000A0044756D704420202020203030E2
:101209002030312030322030332030342030352026
:1012190030362030372030382030392030412030E6
:10122900422030432030442030452030460A0045D2
:101239007272206B657900526420656570726F6DFA
:101249000A005264204D454D0A00526420436F64E0
:10125900650A0044656275674950204F4E0A00448B
:10126900656275674950204F46460A0044656275B4
:101279006755736572204F6E0A004465627567553C
:10128900736572204F46460A0044656275674D735F
:1012990067204F6E0A0044656275674D7367204F7A
:1012A90046460A00436F6E666967206C6F636B215F
:1012B9000A00577220656570726F6D0A00205361CC
:1012C900766520656570726F6D210A00457272201E
:1012D9004D414321004C6F61643E3E002A003C4170
:1012E90030313D003C4130323D003C4130333D001E
:1012F9003C4130343D003C4130353D003C413036C5
:101309003D003C21003C5330313D003C5330323DDF
:10131900003C5330333D003C5330343D003C5330A6
:09132900353D003C5330363D0017
:06340600016900016700EE
:10344F00C2AFC28E438910E4F58B758DB8D2ABD263
:04345F008ED2AF2238
:03001B00022A6D49
:102A6D00C0E0C083C082C0D0C2AFC28E758B00756E
:102A7D008DB820060675A61E75A6E10567D202E57E
:102A8D006960020569E568D3940140021568056C1B
:102A9D00E56C540F7050D20EE56C543F701AD20095
:102AAD0090668DE0601204F0E0D394B4400A9080FB
:102ABD00007480F0C2AF80FE906688E0600204F082
:102ACD00906104E0600214F090668EE0D3940140B2
:102ADD0003E014F0300502056AE56BD394644004FD
:102AED00D2068002056BE566D3940140021566D2CD
:0C2AFD008ED2AFD0D0D082D083D0E03297
:1008B000C20B7D027C007F071233E98F25E525649A
:1008C0006060097D017F6012335DD20BE4FDFC7F27
:1008D0000B1233E98F25E52530E6097D04E4FF128C
:1008E0003381D20B7D017C007F071233E98F25E530
:1008F000257008FD7FFF12335DD20B300B031260B1
:1009000000C2AFC288C2A8C2AA758900122B09D240
:10091000AF90634C7403F0A374CCF0E490634BF09D
:10092000122788123439C206123096906358E0C3F9
:10093000940350037403F0D20BC20DC20CD2932067
:100940000B077E0E7F29122499E4906578F012340B
:100950004FC2AFA37408F09062B77424F0E4A3F020
:10096000906341E09062B9F0906342E09062BAF027
:10097000906343E09062BBF0906344E09062BCF00F
:10098000906345E09062BDF0906346E09062BEF0F7
:10099000756801E490657AF0C207C208C209C20A0C
:1009A000D2AF75A70775A61E75A6E1200B18AF2557
:1009B000FE7D0312259AE4FF1229237E637F78E4EB
:1009C000FB7D0112269490668DE060037401F0E4D3
:1009D000906104F0A37455F0A37481F0E4F56AE427
:1009E000F56B906104E07003121C8C90668EE0B48D
:1009F00001119080007410F0E490668EF0D20BC26A
:100A00000CC20D908008E0F52530E405D207741083
:100A1000F0E52530E508D2099080087420F0E5253E
:100A200030E608D2089080087440F0E56AD3940359
:100A30004023908002E4F0908001F0908000F0E587
:100A40006AD39406400FE4F56AC20390657AF075A4
:100A500068011230969080A0E07003122E2A9080D8
:100A6000B8E07003122EA49080D0E07003122F1E05
:100A7000908000E07013300710122395906334EFDC
:100A8000F0D394004003120036908002E07006908C
:100A90008000E06005D2050209DFC205E4F56A9036
:100AA0006104E060030209DF300912121F839063C2
:100AB00034EFF0D394004005E0FF1234D320080354
:100AC000020C39121E0E906334EFF070030209DF3E
:100AD000906378E054BF247F7003020B9C14700372
:100AE000020B7424026003020BCF200B077E0E7FE3
:100AF00032122499300F74200371906350E0FF701C
:100B000006906354E06055906684E0FEB50722A32A
:100B1000E0FF906351E0B50718906686E0FF9063B0
:100B200052E0B5070C906687E0FF906353E06F607A
:100B30002B906354E06E7033906685E0FF906355B0
:100B4000E0B50727906686E0FF906356E0B5071B87
:100B5000906687E0FF906357E0B5070F90657A7461
:100B600001F01234D9756801020C3990668474FF63
:100B7000F0020C3990668DE060037401F090667CA1
:100B8000E0FF90637AE06F6003020C3990667CE0CE
:100B900004F0E4F568906578F0020C393003030244
:100BA0000C39906347E070030209DF12001ED20384
:100BB000E4F568906578F090668804F0E490667BD0
:100BC000F0A3F0200B737E0E7F40122499806A9070
:100BD000668DE060037401F0300352906378E0208A
:100BE000E74B90637AE0FF90667BE0FE6F600D90CC
:100BF0006683E07007EE146F703F801390667BE0B1
:100C000004F0906334E0FFD3940440031234D69090
:100C100060007482F0A37401F090637AE090600247
:100C2000F07E607F007D03122D2C0209DF300F095A
:100C300020030690668474FFF0200303020CEEE5A7
:100C400068706B123148EF60207E647F7890647921
:100C5000E02404FD122D2C906683E060030209DF7E
:100C6000906358E0F5680209DF906688E0D3943C11
:100C7000403C906683E0703690668804F09062B6DF
:100C8000E0702B12286EE4906478F0A37412F09058
:100C9000667CE090647AF0A374FDF090610763A233
:100CA0000190647C63A2017F121219DA809B1234D6
:100CB000C1EF60159060007483F0E4A3F07E607F64
:100CC000007D02122D2C0209DFE568640160030239
:100CD00009DF906578E004F0E0C394055003020C4E
:100CE00049C203E490657AF01234D90209DFE5685D
:100CF000640160030209DF90657AE014604624FE17
:100D00006042147003020DDC240460030209DFE476
:100D1000F56A200F1390657A7404F0906578E054BA
:100D200001F07568010209DF9080027410F0E49010
:100D3000657AF090657804F07568C890668474FFF1
:100D4000F00209DF906684E07003020DCB906478B6
:100D50007480F090647A7401F0E4A3F0A304F0A32B
:100D60007430F0A3747BF0E4F525747F2525F582BB
:100D7000E43464F583747DF074802525F582E434D1
:100D800064F583E4F0E5252407906479F07C667DC2
:100D90008490634CE0FAA3E0FB7F02122C287E646F
:100DA0007F78E5252409FD122D2C906683E0601BD9
:100DB00012001ED203E4F568906578F0906688040E
:100DC000F0E490667BF0A3F00209DF90657A74048A
:100DD000F0906358E02432F5680209DF90800274D5
:100DE00010F0756803906578E06401FFF090657A13
:100DF0007401F0EF7019906354E06013FCA3E0FD00
:100E0000A3E0FEA3E0FF9066841217C10209DF9001
:100E10006350E0FCA3E0FDA3E0FEA3E0FF90668446
:080E20001217C10209DF80FE78
:010E280022A7
:10003600906379E0B444047F0180027F0090637886
:10004600E0B447047E0180027E00EE5F604A906362
:1000560041E090637AF0906342E090637BF09063B6
:1000660043E090637CF0906344E090637DF090639E
:1000760045E090637EF0906346E090637FF0906386
:10008600797452F09062B063A2019080A863A201D5
:100096007F061219DA0208A6906334E0C39408506A
:1000A600030208AF906341E0FF90637AE06F60035C
:1000B6000208AF906342E0FF90637BE06F6003024B
:1000C60008AF906343E0FF90637CE06F6003020833
:1000D600AF906344E0FF90637DE06F60030208AF7A
:1000E600906345E0FF90637EE06F60030208AF9087
:1000F6006346E0FF90637FE06F60030208AF9063A2
:1001060079E0B444159062B0E0B4FF0E63A20190AA
:1001160080A863A2017F061219DA90668DE060035B
:100126007401F090668E7464F09063797452F09066
:100136006378E0646D60030202B37BFF7A0E794A4E
:100146001213947BFF7A0E7964906341E0F52EA337
:10015600E0F52FA3E0F530A3E0F531A3E0F532A3F7
:10016600E0F533121394752EFF752F0E7530C17599
:1001760031FF75320E7533CD7BFF7A0E799A1213E5
:10018600947BFF7A0E79D61213947BFF7A0F793C13
:100196001213947BFF7A0F7969906347E0F52EA3DB
:1001A600E0F52FA3E0F530A3E0F5311213947BFFC1
:1001B6007A0F7993906350E0F52EA3E0F52FA3E034
:1001C600F530A3E0F5311213947BFF7A0F79C190D5
:1001D6006354E0F52EA3E0F52FA3E0F530A3E0F598
:1001E600311213947BFF7A0F79EF90633DE0F52E81
:1001F600A3E0F52FA3E0F530A3E0F5311213947BCD
:10020600FF7A107912906339E0F52EA3E0F52FA35B
:10021600E0F530A3E0F5311213947BFF7A10792FC5
:10022600906358E0F52E1213947BFF7A10795912D9
:1002360013947BFF7A107982A20FE433F52E121302
:10024600947BFF7A1079B2906683E0F52E121394B0
:100256007BFF7A1079DD90668DE0F52E1213947B84
:10026600FF7A1179109062B6E0F52E1213947BFF97
:100276007A11793EA201E433F52E1213947BFF7AAC
:1002860011796A90667DE0F52EA3E0F52FA3E0F5DF
:1002960030A3E0F531A3E0F532A3E0F53312139471
:1002A6001233A57BFF7A1179B512139422906378E5
:1002B600E0644C70757E117FBB122499906380E0D8
:1002C600F526A3E0F527E4F5297E117FF612249999
:1002D6007D03AF27AE2612259A7E117FF812249948
:1002E600E4F528852782852683E0FF74822528F594
:1002F60082E43463F583EFF00527E52770020526CF
:100306000528E528B410DC7E637F82E4FB7D1012AD
:1003160026947E117FFB1224990529E529C39410A2
:1003260040A77E117FFB12249922906378E0646CCB
:10033600705CF52A7E117FFD122499E4F529AF2A17
:100346007E007D0312259A7E117FF8122499E4F52A
:1003560028A82AE6FF74822528F582E43463F5830B
:10036600EFF0052A0528E528B410E67E637F82E4CF
:10037600FB7D101226947E117FFB1224990529E538
:1003860029C3940840B87E117FFB122499229063FA
:1003960078E0644B7061F528746A2528F582E434A8
:1003A60063F583E06032746A2528F582E43463F5E8
:1003B60083E0F46023746A2528F582E43463F583C8
:1003C600E0FF74802528F582E43463F583E0B50701
:1003D600100528E528B408C09061047432F00208BC
:1003E600A69063787421F0300B030208A67E127F74
:1003F600381224990208A6906378E0B4521A200BAA
:10040600077E127F401224999063787472F07E639F
:100416007F787D08122CAC22906378E064497045A1
:10042600200B077E127F4B122499906380E0F526FD
:10043600A3E0F527E4F528852782852683E0FF7467
:10044600822528F582E43463F583EFF00527E52756
:10045600700205260528E528B480DC7E637F787D5A
:100466008A122CAC22906378E064437079A3E0642E
:10047600527046200B077E127F5312249990638098
:10048600E0F526A3E0F527E4F5288527828526836F
:10049600E493FF74822528F582E43463F583EFF054
:1004A6000527E527700205260528E528B480DB7EAA
:1004B600637F787D8A122CAC22906379E064576062
:1004C600030208AF906380E0F526A3E0F527748267
:1004D6002528F582E43463AD82FC7B80AF27AE2607
:1004E6001232590208A6906378E06444600302055C
:1004F6007D906380E0FF644470030208A6EFB43188
:100506000CC20B7E127F5C1224990208A6906380AF
:10051600E0B4300CD20B7E127F681224990208A632
:10052600906380E0B4320CD20C7E127F751224994F
:100536000208A6906380E0B4330CC20C7E127F835F
:100546001224990208A6906380E0B4340CD20D7E82
:10055600127F921224990208A6906380E0B4350CAB
:10056600C20D7E127F9F1224990208A6906380E036
:10057600FF1234630208A6906104E07013200B0793
:100586007E127FAD1224999063787421F00208A63A
:100596009061047432F0906378E0FFB4510A908061
:1005A600007480F0C2AF80FEEF64577045200B07E1
:1005B6007E127FBB122499906381E0906334F0E44D
:1005C600F528906334E0FFE528C39F40030208A6A0
:1005D60074822528F582E43463F583E0FF90638016
:1005E600E0252824AFF582E43461F583EFF0052891
:1005F60080D0906378E0645360030206AB200B075B
:100606007E127FC6122499906341E0FF9061B8E0A4
:100616006F703C906342E0FF9061B9E06F7030907C
:100626006343E0FF9061BAE0B50724906344E0FFBE
:100636009061BBE0B50718906345E0FF9061BCE0B0
:10064600B5070C906346E0FF9061BDE06F601690C1
:1006560063787421F0300B030208A67E127FD51250
:1006660024990208A6E4F528E4F56B74AF2528F56D
:1006760082E43461F583E0FDAF281232B90528E53E
:1006860028C394FE40E29080007480F0C2AFE490EC
:100696007FF0F0A3F0907FFD74AAF0A374FFF0A39F
:1006A6007455F080FE906378E0644F704C906380E0
:1006B600E0F526A3E0F527E5274526700A200B0777
:1006C6007E127FDE122499200B077E127FE512240C
:1006D60099E4F52874822528F582E43463F583E0ED
:1006E600852782852683F00527E5277002052605DE
:1006F60028E528B480DE0208A6906378E0FFB445BA
:10070600279080007480F0906380E0FDA3E0907FE6
:10071600F0CDF0A3EDF0C2AF907FFD74AAF0A37404
:10072600FFF0A37455F080FEEF646560030208A62F
:10073600906380E0FFA3E0907FF0CFF0A3EFF0E4BA
:10074600F526F527D3907FF1E09527907FF0E09589
:10075600264021E4F56B2527FFE5263478FE7B80CD
:10076600AD27AC2612325974802527F527E43526A5
:10077600F52680D07E127FE7122DACEF4E60201258
:100786000003906347EFF0120003906348EFF01206
:100796000003906349EFF012000390634AEFF07E86
:1007A600127FED122DACEF4E6020120003906350C5
:1007B600EFF0120003906351EFF0120003906352C2
:1007C600EFF0120003906353EFF07E127FF3122DC9
:1007D600ACEF4E6020120003906354EFF01200035A
:1007E600906355EFF0120003906356EFF01200038A
:1007F600906357EFF07E127FF9122DACEF4E60201A
:1008060012000390633DEFF012000390633EEFF099
:1008160012000390633FEFF0120003906340EFF085
:100826007E127FFF122DACEF4E6020120003906304
:1008360039EFF012000390633AEFF0120003906371
:100846003BEFF012000390633CEFF07E137F05123E
:100856002DACEF4E6008122FDF906358EFF0E4F5F1
:1008660028E4F56BE52804FF74392528F582E4347D
:1008760063F583E0FD1232B90528E528C3944340A9
:10088600E09080007480F0C2AFE4907FF0F0A3F0B7
:10089600907FFD74AAF0A374FFF0A37455F080FE58
:0908A6007E637F787D08122CAC02
:0108AF002226
:10322100AE07EEC39430400BEED394395005EE2433
:10323100D0FF22EEC39461400BEED394665005EEAD
:1032410024A9FF22EEC39441400BEED394465005CE
:08325100EE24C9FF22AF0622A2
:103422009062AFE004F070069062AEE004F0906249
:07343200AFE0FF1232E322BC
:10000300123422123221EFC454F0FEC006123422FD
:08001300123221D0E02FFF2280
:102FDF00E4906839F012342290683AEFF0C39430DD
:102FEF004018E0FFD394395011906839E02407F569
:102FFF0082E43461F583EFF08011906839E02407A3
:10300F00F582E43461F583E4F0800C906839E004D4
:10301F00F0E0D3940840BE7531007532007533006F
:0C302F00E4F5347B017A617907121AE89D
:01303B002272
:042DAC008E2B8F2CAF
:102DB0009062AEE4F0A374FFF0123422EF6067F487
:102DC0006064852C82852B83E493B507EC752D0117
:102DD000E52C252DF582E4352BF583E493601E90D8
:102DE00062AFE0252DFF1232E3E52C252DF582E4BC
:102DF000352BF583E493B50704052D80D3E52C2509
:102E00002DF582E4352BF583E49370ADE52D24FF99
:102E1000FFE434FFFE9062AFE02FF09062AEE03E40
:092E2000F07E007F0122E4FEFFB8
:012E29002286
:102788007E137F0B122DACEF4E70037F01227E1358
:102798007F0E122DACEF4E600C123422EF24D024A1
:1027A800FF920F8002D20F7E137F14122DACEF4ED2
:1027B800600C123422EF24D0906683F08005E490F8
:1027C8006683F07E137F1A122DACEF4E600C123424
:1027D80022EF24D090668DF08005E490668DF07E1F
:1027E800137F20122DACEF4E600C123422EF24D050
:1027F8009062B6F08005E49062B6F07E137F2612F0
:102808002DACEF4E600C123422EF24D024FF92013D
:102818008002C20190634163A20190667D63A201B8
:102828007F061219DA30013B7E137F2C122DACEF94
:102838004E603012000390667DEFF0120003906640
:102848007EEFF012000390667FEFF01200039066AF
:1028580080EFF0120003906681EFF012000390669B
:0628680082EFF07F002268
:1031A100906579E0C3947C503D906579E0FE04F030
:1031B10074B72EF582E43462F583EFF0BF0A2790ED
:1031C1006579E0FF04F074B72FF582E43462F5838A
:1031D100E4F0906579E0FF1229CD9065797408F0EB
:0731E1009062B8E004F02247
:103096009080007480F090633963A201F583F58215
:1030A60063A2017F081219DA90634163A20190803E
:1030B6008863A2017F0A1219DA908092E4F0A37461
:1030C60032F0A37401F090634BE0FF9080B1F09072
:1030D60080E1EFF09080957455F0A3F09080007435
:0930E60001F090800974F0F02261
:102E2A00908009E04410F09080A0E0706C9080A13E
:102E3A007482F09080A874FFF0A3F0A3F0A3F07F4F
:102E4A00039080AEEFF07FCBA3EFF07F039080ACCE
:102E5A00EFF0A374CBF09080007402F090682B120C
:102E6A0017CD0000000090682BE0908040F0906839
:102E7A002CE0908041F090682DE0908042F09068BC
:102E8A002EE0908043F0A3E4F0A3F0A3F0A3F09027
:092E9A008018F0A3F0A3F0A3F0EE
:012EA300220C
:102F1E00908009E04440F09080D17482F090634C30
:102F2E00E0FF9080DEF090634DE0FF9080DFF09048
:102F3E0080027402F090682F1217CD0000000090EE
:102F4E00682FE0908058F0906830E0908059F090B3
:102F5E006831E090805AF0906832E090805BF0A388
:102F6E00E4F0A3F0A3F0A3F0908030F0A3F0A3F070
:022F7E00A3F0BE
:012F8000222E
:102EA400908009E04420F09080B8E0706C9080B984
:102EB4007482F07F039080C6EFF07FCDA3EFF07FA4
:102EC400039080C4EFF0A374CDF09080C074FFF041
:102ED400A3F0A3F0A3F09080017402F09068331281
:102EE40017CD00000000906833E090804CF09068AB
:102EF40034E090804DF0906835E090804EF090681A
:102F040036E090804FF0A3E4F0A3F0A3F0A3F09098
:092F14008024F0A3F0A3F0A3F067
:012F1D002291
:102C28008C268D27A907EAFDE975F018A424ACFFC6
:102C3800E5F034808F82F583EDF0EBFDE975F0184F
:102C4800A4FFAEF024ACFBEE34808B82F583A3EDB9
:102C5800F08527828C83E0FDEF24A8FFEE3480FE08
:102C68008F82F583EDF08527828C83A3E08F828E97
:102C780083A3F0852782852683A3A3E0FDE975F069
:102C880018A424A8FFE5F03480FE8F82F583A3A35F
:102C9800EDF08527828C83A3A3A3E08F828E83A384
:042CA800A3A3F022D0
:062CAC008D2BAB07AA0608
:102CB200908000E020E57290682BE0FCA3E0FDA389
:102CC200E0FEA3E0F52F8E2E8D2D8C2CAE02AF03ED
:102CD2008E838F8263A201E52E540744C0F583855B
:102CE2002F8263A201AF2B121A4CE4FCFDFEE52FEA
:102CF200252BF52FEE352EF52EED352DF52DEC3558
:102D02002CF52C908040E52CF0A3E52DF0A3E52EC8
:102D1200F0A3E52FF09080007420F0AF2FAE2EAD1F
:092D22002DAC2C90682B1217C196
:012D2B002285
:062D2C008D26AB07AA068C
:102D3200908002E020E57290682FE0FCA3E0FDA302
:102D4200E0FEA3E0F52A8E298D288C27AE02AF0380
:102D52008E838F8263A201E529540744D0F58385CF
:102D62002A8263A201AF26121A4CE4FCFDFEE52A78
:102D72002526F52AEE3529F529ED3528F528EC35F5
:102D820027F527908058E527F0A3E528F0A3E52949
:102D9200F0A3E52AF09080027420F0AF2AAE29ADAC
:092DA20028AC2790682F1217C11C
:012DAB002205
:022923008F26FD
:10292500908001E030E5037F0022906833E0FCA34E
:10293500E0FDA3E0FEA3E0F52A8E298D288C2790E3
:10294500667D63A201E529540744C8F583852A827B
:1029550063A2017F06121A62E52A2406F52AE435E8
:1029650029F529E43528F528E43527F52790657BF1
:1029750063A201E529540744C8F583852A8263A229
:1029850001AF26121A62E4FCFDFEE52A2526F52A8A
:10299500EE3529F529ED3528F528EC3527F527906D
:1029A500804CE527F0A3E528F0A3E529F0A3E52A67
:1029B500F09080017420F0AF2AAE29AD28AC2790A5
:0729C50068331217C1AF26B1
:0129CC0022E8
:102395009081E0E0F5260526052605260526052675
:1023A50005260526052605260526908010E0F52933
:1023B500A3E0F52AA3E0F52BA3E0F52C9081E1E05D
:1023C500F5260526052605260526052605260526C0
:1023D500052605260526908014E0F52DA3E0F52EAB
:1023E500A3E0F52FA3E0F530E52FB52B08E530B5D3
:1023F5002C037F0022E4F526E52F540744E0F583FE
:1024050085308263A20190637863A2017F08121A66
:102415009290637A63A2019062B063A2017F061273
:1024250019DA906378E0F527A3E0F528E4F526901E
:102435006378E0702AA3E024F8F526E52F540744D5
:10244500E0F58385308274082582F582E43583F5CD
:102455008363A20190637863A201AF26121A92AE3C
:1024650027E4FCFDE5302528F530E52F3EF52FED79
:10247500352EF52EEC352DF52D908014E52DF0A398
:10248500E52EF0A3E52FF0A3E530F0908000744031
:03249500F0AF267F
:012498002221
:101E0E009081E6E0F52605260526052605260526FB
:101E1E0005260526052605260526908028E0F529A7
:101E2E00A3E0F52AA3E0F52BA3E0F52C9081E7E0E3
:101E3E00F52605260526052605260526052605264C
:101E4E0005260526052690802CE0F52DA3E0F52E1F
:101E5E00A3E0F52FA3E0F530E4F526E52FB52B0A28
:101E6E00E530B52C05C208021F68E52F540744F073
:101E7E00F58385308263A20190637863A2017F08A7
:101E8E00121A92906378E0F527A3E0F528E528452D
:101E9E002770099080027410F07F0022906684E013
:101EAE00FFF4602D90637AE06F7076906685E0FFA8
:101EBE0090637BE06F706A906686E0FF90637CE0D3
:101ECE006F705E906687E0FF90637DE06F602280AA
:101EDE005090637AE0906684F090637BE090668524
:101EEE00F090637CE0906686F090637DE09066876C
:101EFE00F0906378E0702AA3E024F8F526E52F54DD
:101F0E000744F0F58385308274082582F582E43526
:101F1E0083F58363A20190637863A201AF26121A40
:101F2E0092AE27E4FCFDE5302528F530E52F3EF591
:101F3E002FED352EF52EEC352DF52DAF2CAE2BAD20
:101F4E002AAC29AB30AA2FA92EA82DD31217B04038
:101F5E00099080027410F07F002290802CE52DF005
:101F6E00A3E52EF0A3E52FF0A3E530F090800274E8
:041F7E0040F0AF265A
:011F8200223C
:101F83009081E3E0F5260526052605260526052688
:101F93000526052605260526052690801CE0F5293D
:101FA300A3E0F52AA3E0F52BA3E0F52C9081E4E070
:101FB300F5260526052605260526052605260526D6
:101FC300052605260526908020E0F52DA3E0F52EB5
:101FD300A3E0F52FA3E0F530E4F526E52FB52B0AB2
:101FE300E530B52C05C2090220CEE52F540744E89D
:101FF300F58385308263A20190600463A2017F0EA2
:10200300121AA8906004E0F527A3E0F52890600C6D
:10201300E0FFF4604590667DE0FEEF6E706EA3E036
:10202300FF90600DE06F706490667FE0FF90600E3C
:10203300E06F7058906680E0FF90600FE06F704C27
:10204300906681E0FF906010E06F7040906682E0E0
:10205300FF906011E06F60048032D2D9906004E099
:10206300702AA3E024F2F526E52F540744E8F5830C
:10207300853082740E2582F582E43583F58363A26D
:102083000190600463A201AF26121AA8AE27E4FCF4
:10209300FDE5302528F530E52F3EF52FED352EF5FE
:1020A3002EEC352DF52DAF2CAE2BAD2AAC29AB3054
:1020B300AA2FA92EA82DD31217B05006E52845271D
:1020C30070099080017410F07F0022908020E52D2C
:1020D300F0A3E52EF0A3E52FF0A3E530F090800107
:0520E3007440F0AF267F
:0120E80022D5
:042499008E2B8F2CCB
:10249D00E4F52DF52E908000E030E511052EE52EAA
:1024AD007002052DD394E8E52D940340E89080004B
:1024BD00E030E50302259990682BE0FCA3E0FDA335
:1024CD00E0FEA3E0F5328E318D308C2FE532FFE545
:1024DD00315407FEE42FF52EEE34C0F52D852E82F6
:1024ED00F5837423F0052EE52E7002052D532DC7AF
:1024FD00F582852D83740AF0052EE52E7002052DCB
:10250D00532DC790634163A201852D83852E826370
:10251D00A2017F06121A4C7406252EF52EE4352DD8
:10252D00F52D852B83852C8263A201852D83852E28
:10253D008263A201121A30E4FCFDFE90682BE0F8D4
:10254D00A3E0F9A3E0FAA3E02FFFEE3AFEED39FD8B
:10255D00EC38FCEF2408FFE43EFEE43DFDE43CFCDA
:10256D0090682B1217C190682BE0908040F0906816
:10257D002CE0908041F090682DE0908042F09068C2
:0C258D002EE0908043F09080007420F05D
:01259900221F
:062694008E2B8F2C8D2D12
:10269A00E4F52EF52F908000E030E511052FE52FA7
:1026AA007002052ED394E8E52E940340E89080004A
:1026BA00E030E50302278790682BE0FCA3E0FDA346
:1026CA00E0FEA3E0F5338E328D318C30E533FFE541
:1026DA00325407FEE42FF52FEE34C0F52E852F82F3
:1026EA00F5837423F0052FE52F7002052E532EC7AC
:1026FA00F582852E83EBF0052FE52F7002052E5308
:10270A002EC790634163A201852E83852F8263A21F
:10271A00017F06121A4C7406252FF52FE4352EF583
:10272A002E852B83852C8263A201852E83852F8299
:10273A0063A201AF2D121A4C7408252DF52DFFE462
:10274A00FCFDFEE5332FF533EE3532F532ED35314A
:10275A00F531EC3530F530908040E530F0A3E531C5
:10276A00F0A3E532F0A3E533F09080007420F0AFD7
:0D277A0033AE32AD31AC3090682B1217C178
:01278700222F
:0229CD008F3F3A
:1029CF00E4F540F541908000E030E5110541E54127
:1029DF0070020540D394E8E540940340E8908000EE
:1029EF00E020E57990682BE0FCA3E0FDA3E0FEA3D7
:1029FF00E0F5458E448D438C42E545FFE544540791
:102A0F00FEE42FF541EE34C0F5409062B763A201AA
:102A1F0085408385418263A201AF3F121A4CE4FCCB
:102A2F00FDFEE545253FF545EE3544F544ED3543CF
:102A3F00F543EC3542F542908040E542F0A3E54383
:102A4F00F0A3E544F0A3E545F09080007420F0AFCB
:0D2A5F0045AE44AD43AC4290682B1217C148
:012A6C002247
:06259A008E2E8F2FAB0511
:1025A000E4F530F531908000E030E5110531E5319A
:1025B00070020530D394E8E530940340E890800041
:1025C000E030E50302269390682BE0FCA3E0FDA336
:1025D000E0FEA3E0F5358E348D338C32E535FFE532
:1025E000345407FEE42FF531EE34C0F530853182E6
:1025F000F5837423F00531E531700205305330C79F
:10260000F582853083EBF00531E5317002053090BD
:10261000634163A20185308385318263A2017F0615
:10262000121A4C74062531F531E43530F53053304B
:10263000C7E52E853182853083F00531E5317002A2
:1026400005305330C7F582853083E52FF00531E53D
:1026500031700205305330C7E535240AF535E435CD
:1026600034F534E43533F533E43532F532908040D7
:10267000E532F0A3E533F0A3E534F0A3E535F090BF
:1026800080007420F0AF35AE34AD33AC3290682B9F
:032690001217C15D
:012693002224
:102B0900E4F526E52604FF1232E374392526F58219
:102B1900E43463F583EFF00526E526C3943F40E3EB
:102B2900E4F526E526247FFF1232E3742F2526F5E6
:102B390082E43461F583EFF0742F2526F582E434BD
:102B490061F583E0FF6003B4FF1D742F2526F5822C
:102B5900E43461F5837420F074302526F582E43479
:102B690061F583E4F080090526E526C3948040B326
:102B7900E49061AEF0F526AF261232E374AF252654
:102B8900F582E43461F583EFF00526E526C394FE6A
:022B990040E515
:012B9B002217
:1033C900E4FDFCC3ED9FEC9E5015E4FBFA0BBB003A
:0F33D900010ABA01F8BB90F50DBD00010C80E4AC
:0133E80022C2
:0D349A004390014390025390FE5390FD2299
:0D34A7005390FD5390FE439002439001228C
:0E348B005390FD439002E5905408FF5390FDCE
:013499002210
:0D34B4005390FD4390014390025390FD2280
:0734CC00AE071FEE70FA22AB
:02328D00AD078B
:10328F00E4FC5390FDEDA804088002C333D8FC3052
:10329F00E70543900180035390FE7F051234CC4322
:0932AF0090020CBC08DC5390FDF8
:0132B80022F3
:10330D00E4FF5390FD7E07439002E59030E00D748D
:10331D0001A806088002C333D8FC42075390FD1E56
:08332D00C3EE6480948050DFC0
:013335002275
:1032B900AB05AA0712349A7FA012328D12348BAF54
:1032C9000212328D12348BAF0312328D12348B12EB
:0A32D90034A77F0A7E001233C922D9
:0232E300AB0737
:1032E50012349A7FA012328D12348BAF0312328DB5
:1032F50012348B12349A7FA112328D12348B123311
:073305000D1234B41234A7CD
:01330C00229E
:023259008B2BBD
:10325B00A2AF921DC2AF85A22C53A2FE8E838F828A
:10326B0005A28C838D827409121AD6E52B53A2FE0C
:10327B0043A220121AD853A2DF852CA2A21D92AF13
:01328B00FF43
:01328C00221F
:1033E900A2AF921DC2AF8C838D82EF121AD643A26F
:0C33F90020121AD853A2DFA21D92AFFFD1
:0134050022A4
:02335D008F26B9
:10335F00A2AF921DC2AFE4F5838D827406121AD606
:10336F00E52643A220121AD853A2DFA21D92AF7FE7
:01337F00014C
:01338000222A
:023381008F2695
:10338300A2AF921DC2AFE4F5838D82740A121AD6DE
:10339300E52643A220121AD853A2DFA21D92AF7FC3
:0133A3000128
:0133A4002206
:1018FF00A907E7FFA805EF93C3966008403B74FC68
:10190F002FFF80F00F08EF93C3966008402B74FBF6
:10191F002FFF80E00F08EF93C3966008401B74FA07
:10192F002FFF80D00F08EF93D3966008400B74F908
:10193F002FFF80C01F1F1F1F1FEF54FEF80303F759
:10194F00E893FC08E893FD08E893FE08E893FF226C
:10195F0009E993C39D6008402974FB29F980F109B7
:10196F00E993C39E6008401A74FA29F980E209E9E5
:10197F0093D39F6008400B74F929F980D319191973
:10198F001919E9C313C313FF22740093F8ECC3981A
:10199F004024701F740193F8EDC3984019701474AC
:0E19AF000293F8EEC398400E7009740393F88B
:1019BD00EFC39840037F00227F0122EDF8E6F00887
:1019CD00A3DFFA22EDF8E0F608A3DFFA22E0A36325
:1019DD00A201F0A363A201DFF475A2002263A201AC
:1019ED00F0A363A20122E0A363A201F0A363A2010D
:1019FD00E0A363A201F0A363A201E463A201F0A33B
:101A0D0063A201DFE175A20022E0A363A2016DFED6
:101A1D00936CFDEE058393FC158363A201DFEA75DC
:101A2D00A200227F00E493A363A201F00F600CA338
:101A3D00E583C2E3F58363A20180EA75A20022E08B
:101A4D00A363A201F0A3E583C2E3F58363A201DFE3
:101A5D00EE75A20022E0A363A201F0A3E583C2E428
:101A6D00D2E3F58363A201DFEC75A20022E0A3634C
:101A7D00A201F0A3E58344F8C2E5F58363A201DF7B
:101A8D00EC75A20022E583C2E3F583E0A363A20116
:101A9D00F0A363A201DFEE75A20022E583C2E4D2BA
:0A1AAD00E3F583E0A363A201F0A3B8
:101AB70063A201DFEC75A20022E58344F8F583E019
:101AC700A363A201F0A363A201DFEE75A20022F9CE
:101AD70022C002C004C00612FFF0D006D004D00214
:011AE70022DC
:10346300BF360BD217E4F547F548F563F564BF376C
:0434730002C2172258
:102F8100C2A9438902906827E0FFF58C8F8A75D921
:102F91000475DA4875DB3175DC4975DD4975DE315B
:102FA100E4F5E9F5F9F5EBF5FB906825E0601675B8
:102FB100EC1075ED10E4F5FCF5FD755F08755D101D
:102FC100755E01801375EC8075ED80E4F5FCF5FD0F
:0E2FD100755F80F55D755E10E4F5EEF5FE228D
:1031E800E4FEAF8CEFFD906826E07003A3E06D600D
:1031F80005122F817E01E5D920E2057E02122F817A
:10320800E58920E105122F817E03D28C75D840759F
:08321800B740D2AED2AFAF0601
:01322000228B
:030033000220E9BF
:0B20E900C0E0C083C082C0D075D008EA
:1020F400C2AF30DC56C3E5EC95EEC3955F5012E5F4
:102104005E25ECF5EC30D70405FC801685FCFC80DC
:1021140011C3E5EC955EF5EC30D70415FC8003851E
:10212400FCFC301724854882854783E590F00548F8
:10213400E54870020547F582854783E5EEF00548DA
:10214400E5487002054753470FC2DC30D9293017E0
:1021540024854882854783E590F00548E548700268
:102164000547F582854783E5EBF00548E5487002AD
:10217400054753470FC2D930DA50E55D700405FCBA
:102184008010E55D25ECF5EC30D70405FC80038573
:10219400FCFCE5495480F546E549C313F5493097FD
:1021A400042480F54920160363498020261A05601B
:1021B400E5605407701253603FE560131313541F16
:1021C400244BF8A649754900C2DA30DB71E55D702D
:1021D4000405FD8010E55D25EDF5ED30D70405FD22
:1021E400800385FDFDE561655C6029E55C5407704D
:1021F40013E55C131313541F2453F8E6F54A201512
:1022040003634AFFE54A139296E54AC313F54A0568
:102214005C535C3FB292301723854882854783E53F
:1022240090F00548E54870020547F582854783E448
:10223400F00548E5487002054753470FC2DBD2AFAB
:09224400D0D0D082D083D0E0326A
:10303C0042415544005245565F54495400CCEEE48D
:10304C00F3EBFC20EFEEE4E4E5F0E6EAE820EFF049
:10305C00EEF2EEEAEEEBE020D3D2CA2D31200A00DC
:10306C00CEEFF6E8E820EDE0F1F2F0EEE9EAE83A2E
:10307C0020000A00FF303CFF30410008040C020A1B
:0A308C00060E0109050D030B070FE6
:10340C0052668F0000000000000000000000000069
:05341C000000000000AB
:10347700EF540F90308693FEC454F0FEEFC4540F00
:04348700932EFF225F
:0334D3008F26221F
:0230EF008F2E22
:1030F100906824E0FF04F074A42FF582E43466F5AF
:10310100837420F0E4FFEFC39D503BE52E75F0037F
:10311100A42480F582E43430F583E493FB740193B5
:10312100FA740293F98F827583001216A7FE9068D4
:1031310024E024A4F582E43466F583EEF00F906870
:0631410024E004F080C050
:013147002265
:10333600742F2FF582E43461F583E0FE6420601675
:10334600906824E0FD04F074A42DF582E43466F55B
:0633560083EEF00F80DAA7
:01335C00224E
:10224D00200B09AF267E007D0312259AE4906824A9
:10225D00F0F526E52675F003A42480F582E43430EC
:10226D00F583E493FB740193FA740293F912168EBD
:10227D007003022394E4F528F529F527742F2527FB
:10228D00F582E43461F583E0FF700302238FE526C8
:10229D0075F003A42480F582E43430F583E493FBD8
:1022AD00740193FA740293F98528827583001216CE
:1022BD00A7FEEFB50608752901052802238AE52931
:1022CD00700302238AEE6003022385AD28AF261228
:1022DD0030EFE52614700302238104600302238F7F
:1022ED00AF27123336742F2527F9E43461FA7B01B9
:1022FD00C0031B8B31753200753300E4F534D00308
:10230D00121AE88F2D8E2C8D2B8C2AE4FFFEFDFCEE
:10231D00AB2DAA2CA92BA82AC31217B0601FAB2D69
:10232D00AA2CA92BA82AE47F207E1CFDFC121710D5
:10233D001217A2906826EFF0E4906825F0E47FB0C4
:10234D007E04FDFCAB2DAA2CA92BA82AD31217B005
:10235D0040309068257401F0AB2DAA2CA92BA82A2A
:10236D007F007EC2FD7C001217101217A290682606
:10237D00EFF0800ED210800AE4F529F5280527022A
:07238D0022890526022260EF
:012394002226
:1034390090682674B8F0E4906825F0C21012224D05
:06344900D21A122F8122AD
:10001E00D2149066A17401F0E4F519F515D218C248
:05002E001C1231E82264
:0334D6008F26221C
:10314800301C53E4906478F0A37409F090667CE036
:1031580090647AF0A37414F0E4A3F09067A463A2D7
:103168000190647D63A2017F081219DAC21C90667F
:1031780091E0FCA3E0FDA3E0FEA3E0FFE4FAF9F888
:10318800EF2401FFEA3EFEE93DFDE83CFC90669134
:093198001217C17F01227F002201
:101C8C0030172DC3E5489564FFE5479563FED3EF08
:101C9C009440EE940040197B087D40AF64AE631213
:101CAC002694E5642440FFE43563540FF5638F6498
:101CBC00301A0512001EC21A201403021E0DE5155F
:101CCC006079201976301205E51A20E00820120DF3
:101CDC00E51A20E0089066A1E004F08054A212B34B
:101CEC009212E516C313F5169066A1E024FD600D63
:101CFC0024FE600E2404700F53167F800F43168051
:101D0C00800A75190F8005D211E4F519E5196002E6
:101D1C001519E51914600C24FB70109066A2E516D9
:101D2C00F080089066A3E516F0D2199066A17401B4
:101D3C00F0E51AC313F51A1515808330197BC219F7
:101D4C009066A3E0FF5480FEEF25E0F054A0FF90D6
:101D5C0066A2E0FD54AA6FF52630D00BEE6004D2DB
:101D6C001C800DD2118009EE7004D21C8002D2119D
:101D7C009067A47410F0E4A3F0A3F0ED540FA3F05B
:101D8C00A37450F0E4A3F0A3F03010199066A3E014
:101D9C0054F0FF1234779066A2E0FEC4540F2F90DB
:101DAC0067ABF080329066A2E0FFC4540FFFA3E053
:101DBC0054F02F9067ABF0801EE5605438655B6083
:101DCC0016E55B24085438F55B131313541F244B8E
:101DDC00F8E6F51A751508301127906699E0FCA302
:101DEC00E0FDA3E0FEA3E0FFE4FAF9F8EF2401FF25
:101DFC00EA3EFEE93DFDE83CFC9066991217C1C233
:011E0C0011C4
:011E0D0022B2
:0B34C100301B05C21B7F01227F002290
:10286E00E4FF0F2407F582E43461F5837414F00F4E
:10287E0074072401F582E43461F583E4F07C667D0F
:10288E0094FEED1DAA0470011CF5828A83E0FBAA5A
:10289E00070F74072AF582E43461F583EBF00EBE60
:1028AE0004E07C667D98E4FEED1DAA0470011CF523
:1028BE00828A83E0FBAA070F74072AF582E434614B
:1028CE00F583EBF00EBE04E07C667D9CE4FEED1D10
:1028DE00AA0470011CF5828A83E0FBAA070F740715
:1028EE002AF582E43461F583EBF00EBE04E07C66DB
:1028FE007DA0E4FEED1DAA0470011CF5828A83E022
:10290E00FBAA070F74072AF582E43461F583EBF016
:04291E000EBE04E005
:012922002292
:1033A5007E307F491224997E307F6C1224997E6687
:1033B5007FA4906824E0FD7B051226947E307F7EF5
:0433C5001224992213
:0334D900C2AE225E
:102BA8000208B0E493A3F8E493A34003F68001F28B
:102BB80008DFF48029E493A3F85407240CC8C3332E
:102BC800C4540F4420C8834004F456800146F6DFFD
:102BD800E4800B0102040810204080903406E47E53
:102BE800019360BCA3FF543F30E509541FFEE493F2
:102BF800A360010ECF54C025E060A840B8E493A3B9
:102C0800FAE493A3F8E493A3C8C582C8CAC583CAE3
:102C1800F0A3C8C582C8CAC583CADFE9DEE780BE9B
:0134210000AA
:10168E00BB010689828A83E0225002E722BBFE025A
:09169E00E32289828A83E493228D
:1016A700BB010CE58229F582E5833AF583E02250F8
:1016B70006E92582F8E622BBFE06E92582F8E22242
:0D16C700E58229F582E5833AF583E493225C
:1016D40075F008758200EF2FFFEE33FECD33CDCCCD
:1016E40033CCC58233C5829BED9AEC99E582984050
:1016F4000CF582EE9BFEED9AFDEC99FC0FD5F0D62D
:10170400E4CEFBE4CDFAE4CCF9A88222B800C1B956
:101714000059BA002DEC8BF084CFCECDFCE5F0CB94
:10172400F97818EF2FFFEE33FEED33FDEC33FCEBCD
:1017340033FB10D703994004EB99FB0FD8E5E4F988
:10174400FA227818EF2FFFEE33FEED33FDEC33FC75
:10175400C933C910D7059BE99A4007EC9BFCE99A69
:10176400F90FD8E0E4C9FAE4CCFB2275F010EF2FAE
:10177400FFEE33FEED33FDCC33CCC833C810D707AE
:101784009BEC9AE899400AED9BFDEC9AFCE899F8E9
:0E1794000FD5F0DAE4CDFBE4CCFAE4C8F9227C
:0E17A200C3E49FFFE49EFEE49DFDE49CFC2258
:1017B000EB9FF5F0EA9E42F0E99D42F0E89C45F08F
:0117C0002206
:0C17C100ECF0A3EDF0A3EEF0A3EFF0229B
:1017CD00A8828583F0D083D0821217E41217E41219
:1017DD0017E41217E4E473E493A3C583C5F0C5833E
:1017ED00C8C582C8F0A3C583C5F0C583C8C582C866
:0117FD0022C9
:10133200E53A242EF8E6053A22782B302402782E5C
:10134200E475F00112185F02168E201DEB7F2ED27B
:101352001D8018EF540F2490D43440D4FF30210B59
:10136200EF24BFB41A0050032461FFE53B6002156D
:101372003B053EE53E7002053D30240D782BE475B9
:10138200F00112185FEF0217FE0231A17403D2249A
:101392008003E4C224F53A8B2B8A2C892DE4F53B99
:1013A200F53DF53EE53B60077F2012136D80F57534
:1013B2003CFFC21EC21DC21FC220C222C223C225BE
:1013C20012133BFF700D3024057F0012137EAF3ED7
:1013D200AE3D22B4255FC2D5C22112133BFF24D0F9
:1013E200B40A00501A75F00A783B30D50508B6FFEA
:1013F2000106C6A426F620D5047002D22080D92484
:10140200CFB41A00EF5004C2E5D22102157ED21EDB
:1014120080C6D21D80C0D21F80BCD2D580BAD22253
:1014220080B47F2012136D201F077401B53B00406A
:10143200F1121332FF12136D0213A6D225D22380AA
:1014420095121332FB121332FA121332F94A4B700D
:1014520006794F7A167BFF201F2EE53B602A7E001D
:101462008E827583001216A760060EEE653C70F040
:10147200C2D5EBC0E0EAC0E0E9C0E0EE1215C5D08B
:10148200E0F9D0E0FAD0E0FB12168EFF60AAEBC0C2
:10149200E0EAC0E0E9C0E012136DD0E02401F9D027
:1014A200E03400FAD0E0FBE53C0460DCD53CD980B6
:1014B200877BFF7A1579C1D21F809C7910800279CF
:1014C20008C223C2258008D2D5790A8004790AC2CB
:1014D200D5E53C047002F53CE4FAFDFEFF1213323E
:1014E200FC7B08201E13121332FD7B10301D0A12E2
:1014F2001332FE121332FF7B20EC3382D592D55089
:1015020013C3E4301D069FFFE49EFEE4201E039DEC
:10151200FDE49CFCE4CBF8C21EEC700CCFCECDCC2B
:10152200E824F8F870F38017C3EF33FFEE33FEEDD3
:1015320033FDEC33FCEB33FB994002FB0FD8E9EBB4
:10154200301E05F8D0E0C448B21EC0E00AEC4D4E91
:101552004F78207B0070C2EAB53C0040BCC0E0126C
:1015620015C7D0F0D0E0201E04C4C0E0C4B21EC033
:10157200F0121356D0F0D5F0EB0213A61218BE14D7
:10158200435314BD5814144C14104214C14F14C9BF
:0F1592004414C94914294314CF5514B34614B354
:1015A1004514B347166F5014182D141C2E143F2BDD
:1015B100142023143D2016582A13D848000014374C
:1015C1003F3F3F00790AA2D5202014302209B910EB
:1015D100020404B9080104A2D52023025001042009
:1015E1001F68921FB53B005034C0E07F20302019A6
:1015F1007F30A21F72237222500F12161EC21FC209
:1016010023C222C2257F30800F302203E9C0E012BD
:10161100136D302203D0E0F9D0E0B53BCC30221776
:101621007F30B9100C12136D7F583021077F7880FD
:1016310003B9080312136D301F057F2D02136D7F4F
:10164100202025F87F2B2023F322921F80CF286EA4
:10165100756C6C2900D21E121332301EF8C21E782E
:101661003B30D50108F60213D82D504349581213C7
:10167100322403B405004001E490166A9312135E0C
:0D168100743A12135ED220753B040214BDB2
:101AE8008B2E8A2F8930E4F53AF539F538F537F534
:101AF80035F536E532453345316012EBC0E0EAC0D2
:101B0800E0E9C0E0AB31AA32A93312186FAB2E0559
:101B180030E530AA2F7002052F14F912168EF53B06
:101B2800C394094007E53BD3940D40E1E53B6420AD
:101B380060DBE53BB42D054336038016E53BB42B4B
:101B480005433601800C74FF2530F53074FF352FBE
:101B5800F52FE53460046410703FAB2EAA2FA9302E
:101B680012168E64306009E534702E75340A8029A7
:101B78009000011216A7FF64786004EFB45813436D
:101B8800360175341074022530F530E4352FF52F01
:101B98008007E5347003753408AB2E0530E530AAAC
:101BA8002F7002052F14F912168EF53BC39461406D
:101BB8000AE53BD3947A5003533BDF74D0253BF5B9
:101BC8003BC3940A400CE53B9411406D74F9253BE6
:101BD800F53BE53BD395345060433601853A3F8564
:101BE800393E85383D85373CAF347E00E4FCFDAB9B
:101BF8003AAA39A938A837121810C8ECC8C9EDC9CB
:101C0800CAEECACBEFCBE4FCFDFEEB253BF53AEE82
:101C18003AF539ED39F538EC38F537AF3AAE39AD34
:101C280038FCAB3FAA3EA93DA83CD31217B05003DD
:101C3800021BA1433604021BA1E53620E003E48021
:101C48002DE53245334531601EAB2EE53024FFF9D2
:101C5800E52F34FFFAEBC0E0EAC0E0E9C0E0AB31C1
:101C6800AA32A93312186FE53630E20774FFFFFE77
:101C7800FDFC22E536AF3AAE39AD38AC3730E1037A
:041C88000217A2227B
:1017FE00BB010689828A83F0225002F722BBFE01CA
:02180E00F322C3
:10181000E88FF0A4CC8BF0A42CFCE98EF0A42CFC77
:101820008AF0EDA42CFCEA8EF0A4CDA8F08BF0A4F5
:101830002DCC3825F0FDE98FF0A42CCD35F0FCEB54
:101840008EF0A4FEA9F0EB8FF0A4CFC5F02ECD3919
:0F185000FEE43CFCEAA42DCE35F0FDE43CFC2286
:10185F00FAE6FB0808E6F925F0F618E6CA3AF6228A
:10186F00BB011A89828A83D0F0D0E0F8D0E0F9D09A
:10187F00E0FAD0E0FBE8C0E0C0F00218ED5016E946
:10188F00F8D083D082D0E0F9D0E0FAD0E0FBC0826C
:10189F00C0830218E4BBFE16E9F8D083D082D0E0F3
:0F18AF00F9D0E0FAD0E0FBC082C0830218F62225
:1018BE00D083D082F8E4937012740193700DA3A3B9
:1018CE0093F8740193F5828883E4737402936860CD
:0618DE00EFA3A3A380DFCD
:0918E400EBF608EAF608E9F62229
:0918ED00EBF0A3EAF0A3E9F022FC
:0918F600EBF208EAF208E9F22223
:00000001FF
